:1000000002780030B402D25202168F758C10D26B77
:1000100002155730B502D25102170B32FFFFFFFF16
:10002000FFFFFF32FFFF020032FFFF35334455561A
:1000300020208520F0E4787FF6D8FD85F02090E838
:1000400000E4F0A374EFB583F874F0B582F3A20373
:10005000920190006D75A0C078007402F208E493DC
:10006000F2A308046023E493F2A30880ED15491479
:100070000025420638073C0946226E0FC21D1D1C92
:10008000FD20920A8C0A7DFFFFC20430961D309736
:100090001A7C14C296209713D29630970EC29720DE
:1000A0009609D297309604DCEAD204D296D2977D94
:1000B000177C4C0D90411275A0807800E493F2A358
:1000C00008B8000205A0DCF4DDF27583F41280604C
:1000D00090F408787775F003128079D200743F129B
:1000E000411190E7FE1241114017F0A3B403004004
:1000F00012124111400BF0A31241114004F0A380F1
:1001000002C20012411174541241111225D3122D52
:10011000457435122D5E121A2950726F6772616D27
:1001200020636865636B73756D202D2D2D2D200068
:10013000E4FBFF900000C3741224B4FC7441341B30
:1001400004FDBC00011DE4932BFBE43FFFA3DCF6A0
:10015000DDF4A3A3E4932B7006A3E4932F600B12AA
:100160002D501220817590FD80FE122076300033D4
:10017000121A294F7665726C6179207265766973FF
:10018000696F6E202D2D2D2D20200090E7FEE0249C
:1001900030A3121A64E02430A3121A64E0121A6425
:1001A00012208B7583F01280607583F4128060904A
:1001B000F418788875F003128079745A12226E74DC
:1001C0001BFD12226E74B4FC12226E9041120DE4DB
:1001D0009312226EA3DCF8DDF6E493A312226EE400
:1001E00093A312226E74A13002027461FE7C007926
:1001F0004012226E12022512228CF7543F09500A37
:10020000F8EEC4440F68D36001C3EC92E303FC0E24
:10021000EE30E2DD90021DEC93F5778011030700CC
:100220000B0000000F7B127A00DAFEDBFC22121AB0
:1002300029546F74616C20706F72747320666F75CF
:100240006E64202D2D2D202000AD770D7A00120A2E
:10025000A112208B7436122D5E1209AFE577B4041B
:1002600000500302035824FD0303FCA20592F77912
:1002700040E70965F054806003757700DCF3121ADB
:1002800029536C61766520636F6D6D756E6963616E
:1002900074696F6E202D2000C3E57760061220760A
:1002A0000203581220817C017940121A2920536CD4
:1002B00061766500AD047A00120AA1E76068F5F086
:1002C000121A292020526F6D3A2000A2F012034426
:1002D000121A29202052616D3A2000A2F112034423
:1002E000121A292020492F4F3A2000A2F21203446B
:1002F000121A29202050676D3A2000A2F3120344FD
:10030000121A292020547970653A200020F70B1228
:100310001A294D554C544900801D121A2950432F5B
:100320004D4143008011121A2920204E6F20726522
:1003300073706F6E73650012208B090CBC04028011
:10034000170202AA4009121A29424144200022122F
:100350001A29474F4F440022E5777008122D577530
:1003600090FE80FE90E865F07437122D5E1209AFA2
:0E03700030030812308C500302040675A0E919
:10037E0079009064007D017C507F007B00E493F354
:10038E00120416A309B9000205A0DCF1DDEF75A079
:10039E00EA79009065007C00E493F579E493F3121A
:1003AE000416A309DCF6121A29436F6E66696720DC
:1003BE00636865636B73756D20202D2D2D2D2000C8
:1003CE009067FEE4932B7027A3E4932F702190E99E
:1003DE0000E0B4011A90E901E0B4231390E902E0C1
:1003EE00B4010C90E903E0B40405122076803012BB
:1003FE0020817590FF122D6B1207E84006122D75A5
:10040E0002037B122D7C80ED2BFBE43FFF220123A8
:10041E0001040005100F2B78101A00002100009027
:10042E00E904E0A2E09238A2E1922490E905E0907E
:10043E00E86EF0A3F090E906E090E86CF0A3F0907F
:10044E00E907E0F57790E908E090E863F090E909B4
:10045E00E090E86AF0A3F090E90AE090E868F0A373
:10046E00F090E90BE0F55F90E90CE0F57690E90D80
:10047E00E0F57890E866F090E90EE090ED00F0304F
:10048E00020990E865E0F57F0225FA128011538982
:10049E00F0438901D28CD2A9D2AF755160755060EC
:1004AE00755A40755940120638306E1F74201285E9
:1004BE0052121A295043206B6579626F6172642063
:1004CE0064657465637465640D0A001207961207FD
:1004DE003C303908121AE7755F12803330251F122F
:1004EE001A170D0A00121A2950532F32206D6F75EC
:1004FE0073652064657465637465640D0A00206E0F
:10050E00031206A0306E05121F9AC25C1280EA1208
:10051E0009B8D268D26E757B00757C0090E857746E
:10052E0006F090E8507400F0A3F0122D86120A34F3
:10053E002001030205F9121A290D0A507265737310
:10054E00200090059E122CEB9005B4122CEB20038C
:10055E00581205671205758056121A17656E746566
:10056E0072206B65790022121A45656E74657220D1
:10057E006F6E206B657970616400223098FDC298B1
:10058E00E5992212308C400122B40702D322C322F5
:10059E00C048697420656E74657220746F20707225
:1005AE006F6365656400932000120567120575126E
:1005BE001A2920746F20636F6E74696E75650D0A4B
:1005CE0000E41241114390032003121205914009D9
:1005DE003098F8120589B40DF2D2D1800E12059121
:1005EE0040093098F8120589B40DF2437DC3C20359
:1005FE00E4124111124111A25D924AC25D12176DB1
:10060E00A24A925D128520B3921B122CD7200015A0
:10061E00121A290D0A5374617274696E67206D6126
:10062E00696E0D0A00C201020AC9C2A8D21F90E863
:10063E008574FAF0E55F540FB40548C2AA1207B1EB
:10064E00C2B2120225D2B3780F1285C17C051202F6
:10065E0025DCFBC2F090F401E030E02654E0790096
:10066E00600279FF5382F8438203E0B900E720F07D
:10067E000AB4FEE1128EE9D2F080DA90ED00F012AB
:10068E00853422B40408C2AA124096D2B3221207AD
:10069E008322206E7575B0FF7A0A7914E5B0543C4A
:1006AE00F8E5B0543C687009D9F7E8542464246026
:1006BE000CDAE9121A290D0A50430080537850D8EB
:1006CE00FE7904B2B27850D8FEA2B413A2B513D9F3
:1006DE00F2D2B2B4CC14755F4412063812073C1233
:0E06EE001A294170706C65008026B488028065
:1006FC0003B4DD18755F5512063812073C121A1731
:10070C000D0A00121A2953756E008006121A295010
:10071C004300121A29206B6579626F617264206341
:10072C0061626C6520646574656374656420002285
:10073C00C225C24DE55FB455061207B1C2AA22B458
:10074C004403C2AA22C24B1207B11209AF121A9764
:10075C00121FDA30390122202514304B19E55F5471
:10076C00F0B4500122E55F540F4420F55F22E55FA1
:10077C00540F4410F55F22752508D288D2A8C2897F
:10078C00D2B2121F5D4002D26E22752608D2BAD2A6
:10079C008AC28BD2AAD2B31209AF121F7A4005D2E9
:1007AC0025121F7A22E55FC4540775F000B40304C8
:1007BC00D2F08005B40502D2F07866C2F190F40054
:1007CC0012807990F4101280791207D922D2EEF1AE
:1007DC00DFC2EE79007A40D9FEDAFC22121A2952D5
:1007EC00656C6F6164696E67204E5672616D207422
:1007FC006F20666163746F72792064656661756CD5
:10080C00740D0A00122D9E1209467B007F0075A004
:10081C00EB790090041C7C00E4BC5000502EBC40D2
:10082C00004008904111EC540F801BBC3000400478
:10083C0074108018BC200040047401800FBC1000A0
:10084C0040047402800693BC0702E577F312041689
:10085C00A3090CBC00C29064001208D6500122906F
:10086C00EB007C007412F0120416A3DCF790650008
:10087C001208D650012290EB007C40E4F0A3DCFB84
:10088C007E08906600BE010E75A0EB793EC3E49B1A
:10089C00F309C3E49FF375A0EB79001215495002DC
:1008AC00D322DEE17B017E40906800C082C083C011
:1008BC00061208FED006D083D08275A0EB79001208
:1008CC0015495002D322DEE3C3227C0075A0EB79DC
:1008DC0000EC2582F582EC29F9C004C082C0831299
:1008EC001549D083D082D0044007EC2440FC70DC46
:1008FC00C322780490EB00D2217C00EC242B83F0F3
:10090C00BC081CBB00067D007A0180048B057A00B4
:10091C00C000C006122092D006D0007C0B8002A32F
:10092C000CBC10D70BD8D2C22122436F6D707574DA
:10093C006572202020202020202090095E75A0EFD9
:10094C007980E493F3A3097409B583F674AFB58287
:10095C00F122C083C08290555574AAF0902AAA74D3
:10096C0055F090555574A0F0D082D083C083C082CE
:10097C00C0017C40E3F0DC02800409A380F6C3F8DC
:10098C00E49368400430E7F8D320E7F4D001D08238
:10099C00D0837C40E493F8E3A309B50004DCF5C3F1
:1009AC0022D32278007900D9FED8FC2274E61222D8
:1009BC006E7C01EC12226E90ED00E0A312226EDC34
:1009CC00F990E9147E04120A2590E9247E14120A87
:1009DC002590EA047E24E578603790E930E0FA85CA
:1009EC0078F0A42404C39578F5827583EA7C0C799D
:1009FC0005EE12226E0EE578B501005005E07A0185
:100A0C008002741212226EE5822AF58209DCE280E1
:100A1C0003120A25E412226E227C0CEE12226E0EB8
:100A2C00E0A312226EDCF422E578B40200402E7CA6
:100A3C0001BC0400C00450098C74741612813B80F4
:100A4C001474011221EDECC41221ED74EF1221ED9E
:100A5C0074161221EDE578D0040CB504D422C0E054
:0E0A6C00C082758205E4D5E0FDD582F9D08206
:100A7A00D0E02275F010A42400F582E5F03468F580
:100A8A008322120A7D5382C075A0EB79007C40E470
:100A9A0093F3A309DCF922300124D22190E810C093
:100AAA0004C001122092C2217C0390E810E0128552
:100ABA0052300003124111A3DCF3D001D0042230DA
:100ACA006B0312156AE55C7013304C05121F9AC24B
:100ADA004C306D0812073C128E7EC26D122DCB90DF
:100AEA00E866E0F578E55F540FB40416D55B347513
:100AFA005B10E5537003123EE9E55C7026123F4530
:100B0A008021B40508121A71121A978016C24B2056
:100B1A003911121A97304B0BE55F54F0B42000508C
:100B2A0002D26D205E0C20700C207109206F060223
:100B3A000B84020D8DE55C6015207209D27290E873
:100B4A003FE4F0803590E83FE0B40200402C7D039A
:100B5A00C27230251574F5121EEC206707121F7A2F
:100B6A0040028006DDEAC225C24DD27F752608857D
:100B7A00595A755C00D25F12176D30195C12228CBB
:100B8A005057F8128EC6120B95804E30E73AB48051
:100B9A0008D268747E1285522230E6175300071273
:100BAA000FC25407B40400502FE054F048F0F5790E
:100BBA00D25D2230E505A2E0921B2230E41AD25C13
:100BCA00128EA9E8540FF0227583E8E575C4540F14
:100BDA004440F582E8F0D2752212864D4003020E97
:100BEA0029307A03020C8C30272B90E850E0F8A3C6
:100BFA00E0C868601E75A0ECE2F556700908B8C036
:100C0A00027800E2F557D27A08B8C0027800E8F014
:100C1A00020C8CC22720766AE550B551028063E542
:100C2A005FB444028022B45502801DA851E6B4F78D
:100C3A0006D211D2148007B4F80EC211D214E551AB
:100C4A0004546FF551020D8D121AB930010F307A22
:100C5A000CE556128F0C7005E557128534102302E5
:100C6A008020E550B5510280F91210A2128ED002EE
:100C7A0020F9E550B5510280F91210A2128ED50260
:100C8A0021B4307B11124111207B08305405121413
:100C9A0000C254020D8D202747207C03020CB1129A
:100CAA002DD7403C020D8D203936307A33E556B4C3
:100CBA004A04D263802AB4CA1230631BE55F540F18
:100CCA00B40504D2538019D2768015B42D09305355
:100CDA0006D276C2538009E4F57A522CC25EC25318
:100CEA00301907307A32C27A805BE5537050307A15
:100CFA0027C27AE55654FCB428258556F090E82098
:100D0A0075552030F10574E0120D2430F00574F0A9
:100D1A00120D24E557120D248069F0A305532230E1
:100D2A001810E556700CE557B41900400512813BBE
:100D3A008045128B35E553603E755520C27A75A001
:100D4A00E8A855E2F830192A122237E556128EC160
:100D5A007001F412226EB4FF08E557A21892E680D9
:100D6A0009E55654FCB4280FE557128EBC12226EC0
:100D7A0080051281C2400C307609E5537005C276AF
:100D8A0002100A307302802BE559B55A02802412E8
:100D9A001D3530011E30731B742012855274751272
:100DAA00855290E82DE0128534A3E0128534A3E041
:100DBA00128534E55C700F307365128CEAE55C606D
:100DCA005E755E28C27375A0E8A95EE3F830194C17
:100DDA0012223790F41A7415F07582187407F0907D
:0E0DEA00E828E0128ECB12226E12223750152E
:100DF800B480127C0390E829E0A3128ECB12226EF5
:100E0800DCF6755C0090F419E030E3FC30E2F99010
:100E1800F41A7415F07582187403F0020E29128200
:100E28001F12814C304F07302622C226C24F105A5B
:100E38004010592A10584F203D54105D75103C0F32
:100E4800105C0F105B12105F12107509020FB702C9
:100E58000ED0020F29020F77020EEE020EF8128E44
:100E6800A95407303905A21BB392E7120F11020FDC
:100E7800B7120FD6203905B40302D23CA23992E743
:100E8800120F11020FB7E576120F11020FB790E893
:100E980077E004F0A2E01403C2E7900FCD93600856
:100EA8004002800874FC8004C23D74F4120F1102E1
:100EB8000FB7203909E55F5407B40400500774F0F0
:100EC800120F11D25A020FB7E579540FB4040280F9
:100ED80003B4050474F88009D23D90E877E4F0740F
:100EE800FAF111020FB774F1120F11D258020FB7AD
:100EF80030251385595A12205874F4121EEC2067B5
:100F080005121F7AC27F020FB7C2267905C0E01208
:100F18001E9DD0E0306605303902D9F1D24FD26A31
:100F280022128EA9F8E55F540FB40407E81240E3D3
:100F3800020FB7B40525C000780E1285C1D000E8AD
:100F4800A2E092F2A2E192F0A2E292F3A2E392F17D
:100F580053F00FA8F01285C1020FB77D0A74ED1285
:100F68000F11303905306602DDF3D259020FB7751B
:100F780083E8E575C4540F4440F582E0F8E55F5412
:100F88000FF9E579540FB404028024B40512B80EA1
:100F980003020F29203912B90515E81285C1800FFF
:100FA800B8ED03020F29B9ED06E8120F118000C24F
:100FB80075205E03020AC902101A7583EAE57644B1
:100FC80000F582E022391911125914765800E57992
:100FD80054077802B4030040027803E55F54FC45E7
:100FE80000F55F30391AE579D2F054F06002C2F0AA
:100FF800E57954077803B404005005A2F092E4227E
:10100800E82290E873E551F0757E00D25E90E8849E
:10101800E4F090E884E0B42003021145C3E55024CD
:10102800109551540FF8E55F540FB4041BB8020033
:1010380040591210A2FE1210A230E74CCE20E74809
:1010480053067F6E7042803BB405234021B80300ED
:1010580040391210A2FE1210A230E72CCE20E72849
:1010680053067F6E70221210A2B47F1C8015B8033D
:101078000040181210A2FE1210A2B4F00B1210A217
:101088006E70051210AF704C02114EE86009A8513D
:1010980086061210AF60F1020AC9A851E6128EE462
:1010A8000853006F885122EE121ABC307A1DC27A9A
:1010B8009011A27C008002A30CE4936016B556F749
:1010C8009011C3EC93B43105200008E422500420A9
:1010D80000F91422BC0A005036E57E75F00AA42CEB
:1010E800500205F0F57E85F07FE52C5407701D054C
:1010F8007AE57AB4020AE577B46300500F02116109
:1011080050FBE577B409005003021161021015BCC9
:101118001100500874F72C422C0210159011E3ECC2
:1011280024F6230493C0E0EC24F62393C0E022C302
:1011380078007908102605D8FBD9F9D322E52C5474
:1011480007700302116190E873E0F551755800E4E7
:10115800F57A522CC25E020D8D12117F4016F57E73
:0E116800E577B57E00400D857E76C238C270F8
:10117600D26FC25DC25C020CE1857FF0E5F0B4027D
:1011860000500CE57E20F005600514C32260FBD3F9
:10119600224410F0A3F0A3EEF0A3F0223031323354
:1011A6003435363738397674706D61777573786B88
:1011B600473B3A43726E69642E0C620F003232323C
:1011C6003232323232323232303030303030323205
:1011D60032323232323232323131323232120F124E
:1011E600141221127A1230124D12611325132A138A
:1011F600FA1345132F1339133D135413BE13AB13B0
:101206008E138413711394139990E868800390E801
:101216006CE57FAE7E121197020CE112117F4051F0
:10122600604FF57712176D020CE1E57F7043E57E9E
:10123600B48000503CC082C08390E863F0D083D075
:1012460082121FC7020CE1E57F7026E57EB402001C
:10125600401F90E930F0D26F020CE1E57F7012E595
:101266007EB41100500BF57890E866F0D26F020C50
:10127600E102114EE57F701FAA7EE57E6019B40B70
:1012860000403EB41400400FB41600400DB41E00DA
:101296004005B421004014020CE1E57EA2E0E55FC2
:1012A600C2E392E3F55FD26D020CE1E55F540FF9FC
:1012B600E57E24EB834501F55FD26D020CE110203B
:1012C60050120FC2BA04047444803EBA0504745521
:1012D6008037BA0B0474668030BA0C0474778029A0
:1012E600BA04004013540FCA24FBB40404740580E6
:1012F60016B405137400800FC4540FA87953000761
:10130600B8040040027401C44AF579D25D120FC2D6
:10131600E579F0FBD24AE582FE12255A020CE1D2AB
:1013260038020CE1C238020CE1D270C238C25DC28A
:101336005C8009D27180F4A201B39201020CE1E54E
:101346002C540760062409FC0211240211612000B6
:10135600031225CD1219C9C238E55FB4440280DCF8
:10136600B4550280D7D24CD26D80D130000AD27CDF
:10137600D27B124111020CE1122ED2020CE1D27B79
:10138600C27C124111020CE1124111020CE1B2249D
:10139600020CE1E579B4550A7400121D1D741E1283
:1013A6001D1D020CE17E009025F4EE936007FA12F3
:1013B6001CFD0E80F2020CE11213C4020CE1E57969
:1013C600540FB40400501120180F201921E574D2CF
:1013D600E212847BE41284B522E57412847B74EFF6
:1013E6001284A4E57412847B74311284A4227431AD
:1013F6001221ED2212140002134212140912147A59
:10140600500022E578606C7B00EB12847BC023C21F
:101416001974EF1284A4EB12847B74151284B5D070
:10142600230BBB04028006E578B503DD22E57824AC
:10143600FC6040FB757540D219D21874011221ED7B
:10144600E5751221EDD22374151221EDE5752410F0
:10145600F575120A6ADBE474161221ED1217F21200
:101466000A6A120A6A120A6A120A6A120A6A120ACE
:101476006AD26F2290E904E0A23820000292E0A22C
:101486002492E1F090E86EE090E905F090E86CE0D7
:1014960090E906F0E57790E907F090E863E090E9D7
:1014A60008F090E86AE090E909F090E868E090E9D1
:1014B6000AF0E55FB444028003B455047412800256
:1014C600C2E090E90BF0E57890E90DF090ED00E0D0
:1014D60090E90EF01209467B007F007C5090E900EF
:0E14E600E493120416A3DCF875A0EB790090D5
:1014F400EA007C00E493F3120416A309DCF690647A
:101504000075A0E9790012154950012290644075D4
:10151400A0E979401215495001229065001208D6BD
:1015240050012290EB007C40E4F0A3DCFB90EB3E06
:10153400C3E49BF0A3C3E49FF09067C075A0EB796C
:101544000012154922128A5112EF8092F0128A2653
:10155400A2F022202B06107E0375250820330610E6
:101564007D0375260832C26B303B12C3E55024104C
:101574009551540FB409005004D2B2C23B303A160C
:10158400C3E5592410955A540FB409005008D2B336
:10159400C23AD249802F90E876104927E004B40873
:1015A400004021755C00E55AB559028016F8E6B48E
:1015B400AA0E0853004FE6700785595AD26D80036E
:1015C40085595AE4F0124111106A11304F0EC24F7E
:1015D400C259C25AC258C25CC25DC25B20393230A1
:1015E40079173077101218B6743112411112411163
:1015F400C277122CD7C279801290E869121666500D
:101604001012188CD277124111800690E8681216D5
:101614005E90E884E004F090E83FE004F012855D19
:1016240020111F201A1C207B1930381690E86D12E7
:101634001666500ED215D270C25DC25C90E86C1270
:10164400165E303F1190E867E004F0B402004006F3
:101654001218E9122FA7122FB422E0A3F0A3E0A3DB
:10166400F022E02410F0501FF84410F0A3A3E0B8D7
:101674000002601314F0B4FF09E81415821582F017
:10168400C3227003E86002C322D322202F1E302B12
:101694000A105272D279D27E152532C55203D2E78E
:1016A400105202C2E7C5521525C22B3210284475C8
:1016B4002508105203D274323013FAC2B2C001C5E5
:1016C4005264FA7008D226C5527930801F64FAC574
:1016D40052A950A7520953016F8950C904546F6528
:1016E400517006D23BC9D00132C97926D9FED2B293
:1016F400D00132C552D21310520520D007800330D6
:10170400D002C213C5523220372030330C10510896
:10171400D279D27DD249152632C55B03D2E7105166
:1017240002C2E7C55B1526C233321030287526087D
:1017340010510132306C31C001A959A75B09530122
:101744004F8959C24BC904544F655A7004C2B3D26D
:101754003AC9D00132C55BD26C10510520D0078044
:101764000330D002C26CC55B32205E27205924208E
:101774005A2120581E203D1B205C18205D15203C5A
:1017840012205B0F10700D107118C26FE577B576DB
:1017940000501B220576E577B5760050117576006A
:1017A400800C1576E5760470058577768000C2078F
:1017B40074AA42C0D21F1289ED12311F20390312BC
:1017C4004111204E031218E91217F2304E0D121A6D
:1017D400172066702A00C218C2192212196712193A
:1017E4002212312610150122301402D25B22A9766E
:1017F400121809F575A2F69219A2F79218A2F59299
:101804004E12869922203904E5787006E9C454F012
:10181400802EE578B40F03E980268578F090E930CE
:10182400E0A414B50100500BC304F5F0E995F025CC
:101834007880DA90E930E0F5F0E984540FC445F09B
:10184400F875F00020390BE854F0C4B57800500264
:10185400D2F7E854C06002D2F6C0F090E930E085D7
:0E18640078F0A4C0E0E5F06006D0E0D0F0E837
:101872002290E865E0D0F025F0C39578B5010050DC
:1018820005D0F0D2F522D0F0E82220180520191C4C
:10189200801FE575C4540312847B74EF1284A4E59F
:1018A20075C4540312847B74021284A4740212213C
:1018B200EDC2EC2220190520180280283019057487
:1018C2000C1221ED30181FE575C4540312847B7489
:1018D200EF1284A4E575C4540312847B740C128441
:1018E200A4201902D2EC22C23F20191F30182EE583
:1018F20075C4540312847B74EF1284A4E575C45436
:101902000312847B74161284A4801230180A74EFB6
:101912001221ED74161221ED74161221EDC2EC2281
:1019220020183C30192F74091221ED12224CD26872
:10193200F854706020C4B40600501AE8A2E7921B63
:10194200128EA9E8540FF0E8C45407F8120FC254DB
:10195200F048F08003120FC2F579D25DD25C2212F8
:101962000FC2F5792220182320190EE575C45403FD
:10197200F57444FCF590D2EC2274011221EDE57568
:1019820054F01221ED740C1221ED222019241219A7
:101992006DE57412847B74EF1284A4E57412847B67
:1019A20074011284A4E57412847BE575540F1284C9
:1019B200A42212197B74EF1221ED74011221EDE5BC
:1019C20075540F1221ED2220181020193A9092A579
:1019D200E574540393457DF57D22301903121A09EB
:1019E200E574540312847B74EF1284A4E5745403E7
:1019F20012847B74301284A4E574540312847BE550
:101A020075540F1284A42274301221EDE575C4546A
:101A12000F1221ED22D083D082E493128552A3E4E7
:101A220093B400F7740173D083D082C082C083E480
:101A320093128552A3E49370F8200007D0E0D0E01F
:101A4200740173D083D082E493B40A02800D300112
:101A52000A300007C001124111D001A3E49370E9DA
:101A62000473300109128552300003124111229091
:101A7200F401E030E01E54E07900600279FF538205
:101A8200F8438203E0B900E7A950F7055053506FBD
:101A9200D27980DB2290F411E030E01A5382F843CD
:101AA2008203E0A959F7128F25055953594FD24B9A
:101AB200D249D27980DF221210A2F8FCAE5F53061F
:101AC2000FBE0402804EBE05028049E55860030243
:101AD2001BEEB8AA06D26E121F9A22B8DF0040345B
:101AE200B8EF16D223D2397430124111757800C280
:101AF2003875770FD26ED22522B8F00475580122BC
:101B0200B8E00475580222B8E1047558042275F051
:101B120000021BBEE55F540FB404069023AF021B04
:101B2200B0B4052BE5795403B4031F90ED00E0B483
:101B320033028016B434028011E8A2E792F0C2E7C1
:101B4200B458077420A2F0021BE490242F805FC3D4
:101B520092F0E55F540390229C7885B403059023AC
:101B620021788EECB50000505393A87920393BB808
:101B720044028003B85533A85F53000FB80A0050DF
:101B82000CB44C02741BB44B21741E801D30241AF9
:101B9200B44C04744E8013B44D04744F800CB44E94
:101BA20004744C8005B44F02744DA2F08006E8A282
:101BB200E7C2E79364FF701C92F0C2F1E55F6479BB
:101BC200540360277428A2F092E0A2F192E1F55644
:101BD2008C57801264FF30E70975560092E7F5577B
:0E1BE200800492E7F556D27A75580022E55835
:101BF000B401028012B40204C2F0800FB40305D213
:101C0000F0021C13021CD3D3021B52E8B4F004757B
:101C1000580322901C4EE4A393A36015B500F7E48B
:101C20009330F0022402F557755600D27A755800A9
:101C300022901C54D2F1787FECB50000508093F5CF
:101C4000567003021BBE30F003435680021BE8129D
:101C50000159020000000000000000000000000028
:101C600000000000004D00004B00000000000000DC
:101C70000000004E000000000000004F00000000C7
:101C80000000001D00000000000000000000000037
:101C900000000000000000000000000000005B00E9
:101CA00000000000000000000000000000005F00D5
:101CB0000000000000000000000000000053005879
:101CC00052000000505157005956000000005500C6
:101CD0000D547E901CF1E55893B500150558E55854
:101CE0009370117A0F121CFD742D121D1D8002D2EB
:101CF0007A755800221477E1F014F0770090E850DC
:101D0000E0F875A0ECEA7C02B42D027C01F208B880
:101D1000C0027800D2E7DCF5E8F0D22722C0E090DC
:101D2000E850E0F875A0ECD0E0F208B8C002780006
:101D3000E8F0D22722E5592410955A540FF8E55FB0
:101D4000C4540FB4040AB80200403F121D8B8038FF
:101D5000400CB805004033121DC6402E802A204B8F
:101D60001F303908E57954F06005800A304D07B816
:101D7000040040168005B80300400F128DC780088C
:101D8000B803004005121E2FD27322A85AE608534A
:101D9000004F885A75F008A2E7B392F0A2E692E7E6
:101DA000F404A2E792F590E82FF0A85AE608530051
:101DB0004F885AA2E692E7A2E792F490E82EF090BC
:101DC000E82DE5F0F02275F008A85AE630E74EF469
:101DD000A2E292F0A2E192F2A2E092F10853004F47
:101DE000E6FE080853004F2690E82EF0EE6630E736
:101DF00001B392F41853000F430040E6FE08085365
:101E0000004F2690E82FF0EE6630E701B392F50818
:101E100053004F885A90E82DE5F0F0C32208530094
:101E20004FC3E559986004E630E7F2885AD322752B
:101E3000F000A85AE630E6530853004FA2E592F0AE
:101E4000A2E492F1A2E192F4A2E392F5A2E092F26E
:101E5000A2E292F3E60853004FA2F292E6C392F296
:101E6000A2F492E790E82EF0E60853004F885AA2B9
:101E7000F392E643F008A2F592E7F404A2E792F5A4
:101E800090E82FF090E82DE5F0F0220853004FC3C2
:101E9000E559986004E630E6F2885AD322128EE9BA
:101EA000128A51303B03D3803D7F3CDFFEC266C2C5
:101EB000B4D2B2A2D0B37C097E0A7F0030B210DF68
:101EC000FBDEF9D2B4D26680DD121F312066171313
:101ED00092B4121F3BDCF2121F31D2B4121F3B121C
:101EE0001F31121F3BC3D2B4128A2622128EFD125A
:101EF0008A51303A0AC23A855A5980F3D3802C7FEE
:101F00003CDFFEC267C2B5D2B3A2D0B37C09121FB8
:101F1000452067171392B5121F53DCF2121F45D2EA
:101F2000B5121F53121F45121F53C3D2B5128A2672
:101F3000227FFF30B204DFFBD266227FFF20B20493
:101F4000DFFBD266227FFF780830B306DFFBD8F9CB
:101F5000D267227FFF20B304DFFBD26722780079AB
:0E1F600008E550B55106D8F9D9F7D322A8519B
:101F6E00E6128EE40853006F8851C322E4F8FE791E
:101F7E0002E559B55A08D8F9DEF7D9F5D322A85A91
:101F8E00E6128EF80853004F885AC322E55F5407B5
:101F9E00B4040040012274FF121E9D30660122120D
:101FAE00113740FA7A017C00121F5D5004DCF9DA19
:101FBE00F7121FC7D25CD25D2274F3121E9D12114E
:101FCE003790E863E0121E9D12113722C225C24DD2
:101FDE0085595A74FF121EEC30670122121F7A4087
:101FEE00687C03121F7A64AA6002DCF7121F7A90D3
:101FFE002017E493601774F3121EEC121F7AE49309
:10200E00A3121EEC121F7A80E9C864500074F212FB
:10201E001EEC121F7A121F7AC24DB45503D239220A
:10202E006002D24D74E8121EEC121F7A7403121E57
:10203E00EC121F7A74E6121EEC121F7A12205874DC
:10204E00F4121EEC121F7AD2252274F3121EEC200B
:10205E006715121F7A7428A8795300F0B8500274CD
:10206E0014121EEC121F7A22121A29474F4F440DDA
:10207E000A0022121A294241440D0A0022121A297C
:10208E000D0A002275A0E87959E4F319F37C10C308
:10209E00ED33FDEA33FA75F002A801430001E23593
:1020AE00E0D4F218D5F0F7DCE675F003A801D3758D
:1020BE00A0E8E230F003088001C4540F500D700AFE
:1020CE0020F20330F10574208003C3443030210424
:1020DE00F0A3800E305608101E08122CF08003124A
:1020EE008552D5F0CA302102E4F022301736C217DD
:1020FE00547FF890E85CE0540FF94400F582758344
:10210E00EAE8F0E9B576048879D25DB90400400DAD
:10211E007440491221EDE01221ED020D8DE812807E
:10212E00B7020D8D30E60990E85CF0D217020D8DE6
:10213E00B4160AD23F90E867E4F0020D8DB4010B9D
:10214E00303F031218E9D21D020C7CB40C08121891
:10215E00B6C21D020D8DB4020812188CC21D020DDE
:10216E008DB415030213FAB431061213C4020D8D89
:10217E00B43007D248C21D020C7CB4080874901209
:10218E001E9D020D8DA2E792F0C2E7B41900401316
:10219E00B43000500EA2F092E7F557755600D27A81
:1021AE00020D8D020D8D301D10540FF576C271C2C9
:1021BE0070C21D12176D020D8D304811C248D26DBE
:1021CE00B40400500B9092A593457DF57D020D8DC4
:1021DE00C0E074301221EDD0E01221ED020D8D2001
:1021EE000209F8202306B4EF03D22322306403FF42
:1021FE008016B40102800CB430028007F85300F050
:10220E00B84004D264FE22FE122237E412226EEE91
:10221E00A22392E7128EDA12226E306407EF128E2C
:10222E00DF12226EC223C2642212224C5009B480E5
:10223E0002D322B48102D322F8120B9580EBC31085
:10224E00681DC000C0017800791412228C4006D897
:10225E00F9D9F77404D001D000300103128552224F
:10226E00C0E075A0F47819E230E2FCD0E0781BF201
:10227E002275A0F47819E230E0FC781BE22290F48B
:10228E0019E020E003C3E42290F41BE0D322FF09FF
:10229E00FF050301020CFF0A080604462FFFFF4C40
:1022AE0048FF4A7131FFFFFF7A73617732FFFF6398
:1022BE007864653433FFFF447666747235FFFF6EC3
:1022CE006268677936FFFFFF6D6A753738FFFF4129
:0E22DE006B696F3039FFFF42436C3F703AFF6F
:1022EC00FFFF40FF3C3BFFFF7C49473DFF3EFFFFAC
:1022FC00FF1CFFFFFFFF45FFFF11FF1417FFFFFF40
:10230C001060121516182E7B0B5E135D5C190EFFF8
:10231C00FFFFFF077DFFFFFFFFFFFFFF012EFFFF0A
:10232C00FFFF462F02FF4A481C7C713103FF4C7A99
:10233C007361773204FF63786465343305FF447648
:10234C006674723506FF6E626867793607FF4D6DED
:10235C006A75373808FF416B696F303909FF4243A2
:10236C006C3F703A0AFFFF40203C3B0B0D4B49473A
:10237C003D3EFF0C0E57580F5651534550FF115907
:10238C0014175552541060121516187B5BFF5F130F
:10239C00FF5E195CFF1B1E2DFF5DFFFFFFFFFFFFA4
:1023AC004E4F1D6173646668677A7863761C627140
:1023BC0077657279743132333436353B39373A3884
:1023CC00303D6F753C6970476C6A406B3F3E4143D2
:1023DC006E6D4246442F45FF2E4A4F481A4C5859B1
:1023EC005756FFFF60FF5CFF5EFF7BFFFFFF5B5FED
:1023FC00FF5DFFFF991011121314151617FF181912
:10240C00FFFFFF050607030809FF0BFF0DFF0EFF7B
:10241C000AFF0CFF0F505254510453025501494D01
:10242C004BFF1FFF9E9C9F9D01020A030B040C0592
:10243C004D06A90708094C560F0D0E58A0A1575967
:10244C002E313233343536373839303A3B2F45500C
:10245C009B5B5C1FA260A3524671776572747975A1
:10246C00696F703C3D514B1718195DA4A553FF4A79
:10247C006173646667686A6B6C3F403E475F141516
:10248C001610A654A77B487A786376626E6D41422B
:10249C004349AE111213AAABAC9A7C4E444F551C57
:1024AC005EFF2D44B1C0B3B4B5B740B9B0B8BB41B1
:1024BC003A424330313233343536373839BF3FC185
:1024CC003BC2C3B2E1E2E3E4E5E6E7E8E9EAEBECC0
:1024DC00EDEEEFF0F1F2F3F4F5F6F7F8F9FA3C3E25
:1024EC003DB6BA2F6162636465666768696A6B6C36
:1024FC006D6E6F707172737475767778797ABCBE05
:10250C00BDAF1B60303132333435363738392D3D61
:10251C005B5D5C3B272C2E2F2008090D1B7E29218F
:10252C00402324255E262A285F2B7B7D7C3A223C87
:10253C003E3F2008090DB576048B79D25D7583EA90
:10254C004400F582E0B503028004D254EBF0EEF9BE
:10255C00121809F920F71F20F60DE9C45403F9EB02
:10256C001280B7D26D8041E9C4540F44401221ED62
:10257C00EB1221ED8032E9C45403F8E9540F4440C6
:10258C00F943038030F60F74EF1221EDE91221EDBF
:10259C00EB1221ED801274EF1225BBE91225BB74EE
:1025AC00EF1225BBEB1225BB204A03123DD222C0F1
:1025BC00E0E812847BD0E0C023C2191284A4D0239B
:1025CC0022121A290D0A00121A2950726F677261B1
:1025DC006D207265766973696F6E202D2D2D2D20FF
:1025EC00553533440D0A0022733533642D0090F0B9
:1025FC00007C07786675F0011280795382F8E582C9
:10260C002408F582BC040390F400DCEC90F41878F8
:10261C0088D2F112807953A8FA121A294469616799
:10262C006E6F73746963206D6F64650D0A00903C66
:10263C0079122CEBE57F0404FC7483122D01902A93
:10264C00EE122D08D20D5389F0438901D28C903CA7
:0E265C0063122CEB902B08122CEB200D0A744D
:10266A002012226E902B048008741012226E902B76
:10267A0000122CEBE57F04B40203E4800503031483
:10268A005403F548754900754A007549007590FC70
:10269A00D2EC200D0512278D80031226F5C2EC120A
:1026AA002903E549654805496014743045491222F1
:1026BA006E7C06794012227FF709DCF980E1054A2F
:1026CA00E54AB46403754A0074C0122D017A00AD5C
:1026DA004AD21ED256122092C2560547E547B46422
:1026EA0008D20C90F8007408F0809FD202B2027BE4
:1026FA0003754640200208122A5D1228F58003124B
:10270A002A6B7C047AFB80097546407C087AFE05B0
:10271A00462002036302FFEABB0406F5C0E5C08057
:10272A000E500844C3F5B0E5B08004F5C8E5C86AA0
:10273A008A003002036300FF55006004A84646F68B
:10274A00E5D8540F60024243E590543C643C600271
:10275A0042447E0475A0F078191228E6E824F8F8B5
:10276A00DEF775A0F478111228E6EA23FA122A0F86
:10277A00DCA50B122A841228D5BB068F300201224F
:10278A000226F7C202122A6B1228D57C047AFB7B36
:10279A0003E41228F580067C087AFE79FCEABB0479
:1027AA0008F5C0E5C0A8C8801B5013F5B0E5B044D1
:1027BA00C37F0012299CBF0101F442408022F5C860
:1027CA00A8C8E5C07F004912299CC84912299CC89B
:1027DA00BF0106F449C8F449C8694241E86942425E
:1027EA00EA23FAEC30E007E92323F9122A0FDCADD9
:1027FA000BBB06A375C00075C800E5D8F4540F607A
:10280A0002F5437C0490F01B785AE8F023F8E5823D
:10281A0024F8F582DCF4C2EE90F403E8F0122A7A86
:10282A001228D57C04785A90F019E030E00F05821E
:10283A000582E015821582B50003C38001D3E54500
:10284A0033F545E58224F8F582E823F8DCDCE54532
:10285A00C333F54590F411E030E00905820582E0C2
:10286A0065006003434501D2EEE590543C643CF5B3
:10287A0044A202920ED202D2EE122A84E590F454B5
:10288A003C643C42441228D590F411E020E70BC284
:10289A00EE122A7AE030E7028003434402C20212AF
:1028AA002A6B1228D5C2B2122A7AA20E9202783A5A
:1028BA00122B2590F401E030E00A05820582E0B48B
:1028CA003A0280034343101228D522E5905403B4F8
:1028DA000307C2EC7590FC8002059022E254F1B421
:1028EA000100B3E54572E433F54522E4F540F541CC
:1028FA00F542F544F543F54522E5415542FD902957
:10290A002F7C045403B40313E493A3FE7F581229C3
:10291A00EAD20FE493524152428001A3A3ED03038A
:10292A00FDDCE0800802FC01F303CF043F902AC6D5
:10293A007C14E5400303540FB40F0D7E007F58D278
:10294A000F902ACE7C118013BC1004E5418005BC8F
:10295A000802E54213FD500D1229A81229EA12298C
:10296A00FFD20F8002A3A3EDDCDE300F051229FF90
:10297A00C20FE54360061229B11229FFE544600738
:10298A00031229D51229FFE54560061229D9122911
:10299A00FF2275F0083340010FD5F0F93322E49392
:1029AA00A3FEE493A3FF22FD30E4077E007F5312C7
:1029BA0029EAED7F42F5F0A2F092E1A2F192E0A2BB
:1029CA00F292E3A2F392E27E0180087F4480027FC2
:0E29DA00507E00135005FD1229EAED0EBE05D9
:1029E800F422E5496006BE000122232324C32E12E7
:1029F8002D01EF122CF022D20F79C0E4D9FEC912B2
:102A08002A0FC9D5E0F622122A414004C2068016D0
:102A1800200613D206100C0F754700B40702B20D3A
:102A280075810702265222C083C08290F800740C78
:102A3800F0D082D08375470022C006C002C001C012
:102A480000C083C08212308CD082D083D000D001E5
:102A5800D002D0062275B0C3E4F5C0F5C8D2EE1294
:102A68002A842275B0FF74FFF5C0F5C8C2EE122A99
:102A7800842274127900D9FED5E0FB227C0875A067
:102A8800F07802BC040775A0F47802800ABC03023F
:102A98008025BC010280207402F220020474708038
:102AA800027460F27445F2122A7A18E230E00708DC
:102AB80008E2181880F508E82408F8DCC622003770
:102AC800003900380041024102390141013903410E
:102AD8000339044104390238023701380137033811
:102AE800033704380437433132333435363738390D
:102AF8003031323334353600804F5000804C42003C
:102B0800C02030004C4F4F50004F50454E000D0A2A
:102B180000205041535300204641494C00C3122B1A
:102B2800377C08E813122B37DCFAD3122B3722CA6A
:102B3800858AF020F7FA858AF030F7FAB392B285E1
:102B48008AF020F7FA858AF030F7FA858AF020F7BC
:102B5800FA858AF030F7FACA22E4936006A3128550
:102B68005280F622E549600B902C327C0423230422
:102B7800FD8019902B11200D03902B0C122B6190C6
:102B88002B16122B61902C167C057D00E57FB40175
:102B9800021C1CC083C082C001C004C0057A00D2D8
:102BA8002190E810122092C22190E811122B61D0D6
:102BB80005D004D001D082D0830D7907C3E493A354
:102BC800F8E493A3566024400FC083C082902B1F63
:102BD800122B61D082D083D37420128552E493A340
:102BE800128552E493A31285528002A3A3D9CE4042
:102BF8000CC083C082902B19122B618004C083C043
:102C080082902B16122B61D082D083DC862240045E
:102C180030374010303840083039402031304402D5
:102C280031334501323543105131420830374204BF
:102C380030384108303941043130430231314404DD
:102C480031334502323542013037420230384101D2
:102C580030394102313043013131440831334504C0
:102C68003235422030374210303841203039411057
:102C78003130430831314410313345083235428010
:102C88003037424030384180303941403130430498
:102C98003131442031334510323590F8007430F02A
:102CA8007406F0740CF02290F800740DF02290F87D
:102CB80000740CF02275A0F87900F30975A0F87972
:102CC80001E493A36008B45C02748CF380F32220BF
:102CD8007710903CBB201B03903CD1122CEBA21B1D
:102CE800921C22E493A380CD75A0F87901645C60FE
:102CF80004645C8002748CF32275A0F87900F322D6
:102D080075A0F87901E493B45C02748CF3A3DCF544
:102D1800227480122D01E576122D3C7420122CF0BD
:102D28007A00AD760DBD00047A017D00D2561220DE
:102D380092C25622120A7D7C10122D082290F40F9E
:102D48007403F090F41FF022903C8F122CEB229029
:0E2D58003CA5122CEB22C0E07493122D01D08A
:102D6600E0122CF022903C4D122CEB122DB022904A
:102D76003BF5122CEB22903C21122CEB122DB022AB
:102D860090312D12327FD21690E85F7479F090E878
:102D96005E12302E1231DB22903C37122CEB903C27
:102DA60063122CEB74C0122D0122903C0B122CEBFB
:102DB600122DC212308C50FBB407F82212308C4010
:102DC600FB123DC922305708C25720390312335D22
:102DD60022E5536002D322307A10AE56BE2E0EC2C2
:102DE60010C27CC2507C2D122F26022EC320104208
:102DF600BE79217C22122F26C250D21090E8377459
:102E060001F090E838E0123D967C107420F0A3DCC7
:102E1600FC022EC3BE6ED390E838E004B57702807C
:102E2600034001E4F07C2D122F26122EE7C27A020F
:102E36002EC77445A879B855027451B5061390E8A3
:102E460037E0B40102807614F0123D967420F0D378
:102E560022BE4718123DB3C21090E838E0B576039B
:102E6600122D1990E837E0240AFC80BBBE4804D234
:102E760050D322BEC804C250D322BE8000503CBEEE
:102E86002E004039BE4800500E903E5830500390F8
:102E96003E72EE93FE8011BE7B005021BE61004063
:102EA6001CEE30500324E0FE90E837E06411600D1C
:102EB600123D96EEF090E837E004F0D322C27AC3D2
:102EC60022E4F52CF57AC25EC253D322D27C90E876
:102ED60038E576F0C2507A48121CFD122EE7022E13
:102EE600C790E838E0FF903D49122F50D221EF24D9
:102EF60001FDE43400FA90E83B122092E4F090E8F9
:102F06003B122F50C221903D4E122F50EF120A7DD8
:102F16007C10122F60EF120A8C903D52122F502215
:102F260090E850E0F875A0EC7445AB79BB55027497
:102F360051F2D2E708B8C0027800F2C2E708B8C07A
:102F4600027800DCECE8F0D22722202104E493800A
:102F560001E06005122F6E80F122202104E49380A7
:102F660001E0122F6EDCF322C083C082903E0793ED
:102F7600FA53027F20E70C305013C25074C8121D5A
:102F86001D800A205007D2507448121D1DC004121D
:102F96001CFDD004D082D083A322903D80122CEB5E
:102FA60022903D6A122CEB903C79122CEB222011D8
:102FB60069201A41203E02801090E853E0B41E00BA
:102FC6004005123171800204F0201A2920191330AD
:102FD600180A123E05A2E7B3921B8006123E13B3EF
:102FE600921B201C05301B0D8003201B0830390264
:102FF600D25C122CD71230479257501E90E853E4F9
:10300600F0D27990E85F7479F090E85E30221990FA
:10301600F800740CF0C257C2222290E85DE014F06A
:10302600701EA3E014F070187404F015827484F016
:1030360090E85FE014F0700890F8007408F0D2226F
:103046002212308C4008C20690E856E4F0229030F6
:10305600DF9360F214FE3006028004D3D20622BE4D
:103066000B02800DBE0C028008BE0E028003BE0F4E
:103076001390E856E00430E30A2408B4280050DB35
:10308600F080D8F0C32275A0F47583F4780D791D0D
:1030960075820E7A011230CCB40F2975820E7A022F
:1030A6001230CC2410B41F1C75821E7A011230CC4B
:1030B6002420B42F0F75821E7A021230CC2430B42D
:1030C6003F02C322D322EAF0E25403FEE354032371
:0E30D6002342060582EAF0EE22000000000010
:1030E40000000E00000008000502000000000000BF
:1030F40000000100000009000603000000000000B9
:1031040000000F0000000A00070400000000000097
:103114000000100000000D000C0B00201A03122DFB
:103124001922201A03122CD722BE0B0BD270D215EF
:10313400C26FC2380231D4BE0C0BD271D215C26F29
:10314400C2380231D4BE0A2290E835E4F012333991
:10315400903CE7122CEB122CB6D21AC26FC271C289
:103164007090328E12327F0231D4BE0D15C23EA849
:103174001F1231EA403B122CB67491122D01122D0C
:103184002822BE0A004006203E0302322CD23EC250
:10319400381236D1122CAFE51FB43D09E577B4637C
:1031A40000500D800C500AE577B4090050028001EC
:1031B40022C23E1232114007B57702800740051241
:1031C400317A800CF576C270C271C238D26FD215D2
:1031D4001231DB122CB622E490E853F0A3F0A3F0F2
:1031E400751F3BC23E22B83B02C3227E0090E83BDF
:1031F400E0CE75F00AA42E500205F0FEA318B83BE9
:10320400EF90E854F0FDA3E5F0FAF0D32290E855EE
:10321400E0F5F0B40200500E90E854E020F00560B0
:103224000514C32260FBD322C23890E854E576F03B
:1032340090323A12327F90E854E0BE0D0DD26FD234
:1032440015F57690312D12327F22BE0E0814B4FF8C
:1032540010E577800CBE0F1904B577028003400196
:10326400E4F0AF76F57674C0122D01122D1E8F7620
:1032740022122CD790312D12327F22C083C082902B
:10328400E85AD0E0F0A3D0E0F02290E835E0F8BEB0
:103294000B0704B40E0CE48009BE0C2614B4FF0220
:1032A400740DA95F530107B40D05B905E28010B48C
:1032B40004028008B40C028003B40B03B902D0F0FA
:1032C4008073BE0A58105415C21A90312D12327FE1
:1032D4001231DB122D19122CD7122CB622903CFD80
:1032E400122CEB903D13122CEB9032F912327F909A
:1032F400E835E4F022BE0B028003BE0C1290E835E0
:10330400E0F4F0903D296003903D2E122CEB22BE98
:103314000DFC90E835E070B012140080ABBE0DBC1B
:10332400E823F890393B93F9A3E893F58289831253
:10333400327F02335D90E835E0F875F014A4240A76
:10334400F582E5F0343AF5837480122D017C141271
:103354002D081233681233712290E85AE0C0E0A3BA
:10336400E0C0E0229039BFE893122D012290E835A5
:10337400E0FC903975230493C0E0EC2393C0E02271
:10338400903C63122CEB903B22122CEB90E835E03E
:10339400F89039907C00E4A39370030C80F8ECB5AA
:1033A40000F4122CC47429122CF074D3122D0112BF
:1033B4002CAF1231DB9036D112327F22903C631253
:1033C4002CEB903B2E122CEB74C9122D011233718D
:1033D40090373112327F22903B39122CEB903B62B2
:1033E400122CEBE57612352F74C4122D01E57612FA
:1033F4002D3CE576120A8C7490122D01122CAF909C
:10340400E837E4F090E836E4F090E838E576F090B8
:10341400341A12327F2290E837E0FFBE0F080FBF44
:10342400110D7F008009BE0E221FBFFF027F109086
:10343400E837EFF070097490122D01740D800724A1
:10344400C3122D01740E90F800F022EF7036BE0BFB
:0E3454000A1234B804B50010E4800DBE0C5E00
:103462001234B814B4FF03E50014F090E838E0FF1A
:1034720012352F74C4122D01EF122D3C7490122DAF
:1034820001EF120A8C22BE0B0B123D9604B47E1081
:103492007420800CBE0C27123D9614B41F02747D5A
:1034A200F0F8122CB6E8122CF0EF24C3122D01749E
:1034B2000E90F800F022A8770890E838E022BE0AC1
:1034C20013122CB67480122D017C14903A82122DA4
:1034D20008023759BE0D1990E837E06013123DB368
:1034E20090E837E4F07490122D01740D90F800F01A
:1034F20022903B39122CEB903B4C122CEBE57612CE
:10350200352F120FC212353C120FC212355574906C
:10351200122D01122CAF90E837E4F090E836E4F077
:1035220090E838E576F090358312327F22C0E0745D
:1035320091122D01D0E012379322780E540F14F518
:10354200F074C3122D011236841236AF90E839E5B9
:10355200F0F022F8540FB40400400824FDF5F0788E
:1035620003800CE8C4540F9037C393F5F0780474C9
:10357200CA122D011236841236AF90E83AE5F0F005
:103582002290E837E0FFBE0F080FBF030D7F0080D7
:1035920009BE0E381FBFFF027F02BF020990E83941
:1035A200E0B4030050E090E837EFF0122CB6903D03
:1035B200E8E493600B122D01741D122CF0A380F12C
:1035C200903DE8EF93122D01122CAF22BE0B0A128E
:1035D2003DEC04B50010E4800DBE0C4B123DEC1422
:1035E200B4FF03E50014A982B9380AC0E0123651CB
:1035F200D0E090E838F090E838E012352F90E837C4
:10360200E0700E90E838E07583EA4400F582E080CD
:103612000312365FC0E012353CD0E012355590E817
:1036220037E0FF1235C222BE0A1C90E837E0700371
:10363200123651122CB67480122D017C14903A6EFF
:10364200122D08023759BE0DDD90E837E0D2541230
:10365200365FFB90E838E0FEC24A02254290E83924
:10366200E090366D93B444004006220102034455B3
:10367200F890E83AE09038949354F0482290E83574
:10368200E0F89039CEE89390E830F09039DDE89395
:1036920090E831F09039ECE8230493F9E823939011
:1036A200E833F0A3E9F02290E832E0F5F090E83058
:1036B200E0FCC0F0A4D0F0F990E830E0FC90E833F0
:1036C200E0F8A3E029F582E438F583122D0822A858
:1036D2001FBE0A00500F75A0E8EEF208B83F13189B
:1036E20018F208800DBE0E028003BE0F3218B83ADF
:1036F2000108881F7491203E0274D1122D011231EB
:10370200EA400A903C647C03122D088007D25612CC
:103712002092C2567493203E0274D3122D0122BE0F
:103722000A028033BE0DF71231EA403E02392A9076
:10373200E831E0F890E832E0BE0B0704B5000CE493
:103742008009BE0C0F14B4FF02E814F074C9122DE4
:10375200011236A9BE0A10903CE7122CEB122CB6CD
:1037620090328E12327F22BE0D1B90E835E0F8B403
:1037720000028002D25490395993E8230493C0E0A6
:10378200E82393C0E022E4A23892E0FC023827E565
:10379200772401FDE43400FA023833E55F540FB4B4
:1037A20002057C00023827B404047C018077B4054A
:1037B200F17C028070E55FC454079037C393FC80AC
:1037C2006400000103000290E86EE0FD90E86CE006
:0E37D200FA53020F805B90E904E0FC804890FF
:1037E000E86AE0FD90E868E0FA53020F804590E84F
:1037F00063E0F4541FFD7A00D21E803790E863E046
:10380000F4546003C4FC801F90E930E0FD7A00D2DC
:103810001E802090E866E0FD7A00D21E801590EDB3
:1038200000E0FD7A00800C12367F90E832ECF01256
:1038300036A922D256122092C256C21E2290E832D7
:10384000E0A2E0923802392412321140046002F5FD
:103850007702392490E832E090387A93F9540FB423
:103860000209E55F540FB40202A95F895FC000122C
:10387000063812073CD00002392412445590E83231
:10388000E090389493F55FF9895FC00012073CD04F
:10389000000239241222523290E855E090E86CF090
:1038A000A3F090E854E090E86EF0A3F0807690E802
:1038B00032E090E904F0806C90E855E090E868F020
:1038C000A3F090E854E090E86AF0A3F0805690E806
:1038D00054E0F4541FFC90E863E054604CF08044E2
:1038E00090E832E0F4540323C4FC90E863E0541FF2
:1038F0004CF0803090E854E090E930F0802690E879
:1039000054E090E866540FF0801A90E854E090ED8F
:1039100000F0FEC000E412226E740312226EEE125A
:10392000226ED000123368123371122CB6903CE72D
:10393000122CEB90328E12327F222233C03384332A
:10394000C033C033C034F333DB3384338433843344
:1039500084338433C033843384383D389838AE3868
:1039600054387D393A393A384838F438FE38B8385E
:10397000CE38E0390A378837C937D8379D37B73955
:103980003A393A37913808381337DF37EE37FC3891
:103990001E00312D393939000000000000322D326F
:1039A000353600312D313600312D313600312D398B
:1039B000393900322D33300000302D323535008B4F
:1039C0008C8F8A87D4D48F919191928A91D403005D
:1039D000030A0A00000000000000070003020002C2
:1039E0000304000000000000000400053BC40000C8
:1039F0003BBE3B783B96000000000000000000004A
:103A0000000000003BCA00003BE65363616E206D7E
:103A10006F64651D2020202020202020202053635B
:103A2000616E2074696D651D2020202020202020DB
:103A30002020506F776572206F6E207363616E1D5A
:103A40002020202020204B6579626F6172641D2048
:103A5000202020202020202020204D6F7573651D00
:103A60002020202020202020202020202020435003
:103A700055206B6579626F6172642F6D6F75736528
:103A80002020435055206E616D657320202020203A
:103A90002020202020204D6178696D756D20706F89
:103AA0007274731D202020202020457870616E7371
:103AB000696F6E2077696474681D20202020457826
:103AC00070616E73696F6E20756E6974731D20204E
:103AD0002020566964656F20626C616E6B2074698A
:103AE0006D651D2020204B422072617465206B653E
:103AF00079732F7365631D2020204B422064656C11
:103B000061791D2020202020202020202020537596
:103B10006E206B62206C616E67756167651D202089
:103B20002020C04E65772076616C75652800C04303
:103B3000686F6F73659E9F20008043686F6F736529
:103B4000209E9F7F7E20204350551D00C04B421D6C
:0E3B5000202020204D531D202020202020204A
:103B5E0020202000C04E616D6520202020202020D6
:103B6E002020202020202020200050432020202014
:103B7E00202020204D6163202020202020205375FE
:103B8E006E2020202020202050532F322020202055
:103B9E0020205365724D6963736F6674536572505E
:103BAE00436D6F757365536572204F74686572202F
:103BBE004E6F205965734F66664F6E20536C6F774C
:103BCE002020204D656469756D2046617374202038
:103BDE0020466173746573745043315043325043C1
:103BEE00334D616353756E805265736574207375C2
:103BFE00636365737366756C2020202000C048696E
:103C0E007420656E74657220746F2070726F6365B8
:103C1E00656400805265736574206661696C6564C5
:103C2E0020202020202020200080436F6E666967B0
:103C3E0075726174696F6E20726573657420008091
:103C4E00436F6E66696775726174696F6E2062612B
:103C5E006420202000C02020202020202020202092
:103C6E002020202020202020202000802020202006
:103C7E002020202020202020202020202020202036
:103C8E0000C050726F6772616D20636F72727570D3
:103C9E0074656420202000C0536C617665206C69C9
:103CAE006E6B2062616420202020202000C053749F
:103CBE00617475731D206E6F726D616C20202020F3
:103CCE00202000C05374617475731D206E6F2063C5
:103CDE00707520706F77657200C0456E746572A541
:103CEE0073656C656374209E9FA56974656D008015
:103CFE005361766520636F6E66696775726174696C
:103D0E006F6E202000C0456E7465722063686F6907
:103D1E0063659E9F20596573202000CF59657300FF
:103D2E00CF4E6F2000805363616E206D6F646520EF
:103D3E0020202020202020202020004E616D6500B4
:103D4E00203D2000204368616E676520592F4E2F5D
:103D5E004553433F20004F6E204F6666C05374613B
:103D6E007475731D206E6F742073656C6563746556
:103D7E006400C05374617475731D20766964656F39
:103D8E00206F66662020200090E838E05403C4F8C7
:103D9E0090E837E014540F42007583EB7400543FE3
:103DAE0048F582E02212094690E838E0120A7D5367
:103DBE0082C075A0EB79001215492278007900D9DE
:103DCE00FED8FC2290E837E4F0FF123DDC22903D55
:103DDE00E8EF93122D01122CAF2290C2C900BF0141
:103DEE0007780590E839E022780490E83A5006A862
:103DFE00770890E838E022E575C4540F4410F58238
:103E0E007583E9E022C0E0740925748355D8D36028
:103E1E0001C3D0E0220201080444B1C0B3B4B5B767
:103E2E0040B9B0B8BB413A42433031323334353603
:103E3E00373839BF3FC13BC2C3B2E1E2E3E4E5E646
:103E4E00E7E8E9EAEBECEDEEEFF0F1F2F3F4F5F67C
:103E5E00F7F8F9FA3C3E3DB6BA2F616263646566C7
:103E6E006768696A6B6C6D6E6F707172737475765C
:103E7E007778797ABCBEBDAF1B60303132333435C2
:103E8E00363738392D3D5B5D5C3B272C2E2F2008B5
:103E9E00090D1B7E2921402324255E262A285F2B0F
:103EAE007B7D7C3A223C3E3F2008090D2030362F88
:103EBE0031302F393820436F7079726967687420FA
:0E3ECE00313939302D3139393820526F736552
:103EDC0020456C656374726F6E69637320C2A9129E
:103EEC0090C175F02C123FCA123FEB124010200803
:103EFC003F123F97403AD20ED279A950A7060953E8
:103F0C00016FA707B7FF02800EB7B607E506B4B678
:103F1C000280040953016F895030011474201285FA
:103F2C0052744B128552E506128534E5071285341E
:103F3C001290CE128A26D2A922128A51C2A91290AC
:103F4C00C175F03C123FCA123FEB124010200832F0
:103F5C00123F97402DD20DD279A959A706095301CA
:103F6C004FA7070953014F8959D249300114744D99
:103F7C00128552E506128534E50712853474201239
:103F8C0085521290CE128A26D2A922124020402DA0
:103F9C007D081240204026300903C38001D3E5067A
:103FAC0033F506DDED7D081240204011300903C3C6
:103FBC008001D3E50733F507DDED1240202253B025
:103FCC00CB7C92000000DCFB43B0347C1ADCFEE5B9
:103FDC00F07D083312406E0000000000DDF5225326
:103FEC00B0CB7C1FDCFE43B0347C0DDCFE20B40275
:103FFC008004C208800D7CFF20B406DCFBD2088054
:10400C0002C20822C2087C3F30B406DCFBD2088016
:10401C0002C208227CFFDC02801D20B4F97C000C5B
:10402C0030B4FCC3EC940E500AC3EC94034008C2A9
:10403C00098002D209C322D3227C26DCFE227D1009
:10404C00C5F0D312406E0000000000000033124097
:10405C006EBD0904C5F08003000000DDF0C3124002
:10406C006E22C0E053B0CB7C0D500280027C1BDC76
:10407C00FE43B0347C13500280027C05DCFED0E0A1
:10408C00227C127DFFDDFEDCFA22128A51C2A912BB
:10409C0090C175F02B123FCA123FEB12404575F0E0
:1040AC006275E00312404A1290CE128A26D2A922DF
:1040BC004300F830E0055300FB800343000430E17B
:1040CC00055300FE800343000130E2055300FD80E0
:1040DC0003430002E500221240BC85E0827583FF99
:1040EC00128A51C2A91290C175F02A123FCA123F0E
:1040FC00EB1240458582E08583F012404AC20C12D7
:06410C0090CED2A9222290
:1041120002974C32FFFFFFFFFFFFFF758C10D26B3F
:10412200327583F011607583F411601286997900FB
:104132007583E8E92480F582E07583EAF582E0126E
:1041420080B709B904EA90F400786675F000E55F7B
:104152005407117990F410117990F408787775F07A
:1041620003117990F41A7415F07582187403F02211
:1041720075821274C0F075820FE075821FE075823D
:10418200047470F0758214F022438202741AF0F003
:104192005382F8438200741330F2027407A2F09241
:1041A200E0F07407F05382F8438201E8F05382F89A
:1041B200438202748020F1027490F074A020F10214
:1041C20074B0F07405F022C4540F75F0007866B430
:1041D2000500401AB4050575F0018012B406077592
:1041E200F00578668008B407F375F0017899758355
:1041F200F0E9C403F58212807922E590543C537DA4
:10420200C3427D227583F030E3037583F4C4032433
:1042120001F582E030E20D5382F8438203E8F012A6
:104222008F11C322D3755D0022E8B57800401B9040
:1042320092A193FE55906004EE427D22EE557D6080
:1042420009E8784D11F4EEF4527D22F9E574917B80
:1042520074EF91A4E574917BE991A42279387B30C3
:10426200D255E95403C074F574B120D07450028061
:1042720053E578601BE95403F8B5780050028034A6
:1042820090E930E08578F0A428C39578F58280071C
:10429200E954032400F5827583EAE05407B4070564
:1042A200128356801FB40402801A40045195801470
:1042B200E0C45407D1CA430104D1CA5301FBE954F3
:1042C20003F83119090B309803128A8CB93C93C256
:1042D2005522128E80128520204E4940472002032B
:1042E20020182BE5795407B40707E5741280F4808F
:1042F2002AB4041175F0FF128F4C50280554E5546E
:10430200B40A2A801F4007E57412858F8016E5746F
:1043120012847BE890E885F01284B550070554E5D5
:1043220054B4A00975540005551553C322D3221263
:104332008520204E685002806420020320183DE54B
:1043420079C45407B4041888F009E3F8128F635053
:104352000A055DE55DB40A4C755D00755C0022409E
:1043620011B40707E5741285FF8032E5741280F4F8
:104372008022B40207E5741280F48018E5749092EA
:10438200A593557D6017E574D2E212847BE812840E
:10439200B5500A225007055DE55DB4A007755D00C2
:1043A200055E155C22E754036002801AE954031289
:1043B20083A0400122B71005770051B822B4013919
:1043C20077037E0051B880737583E9E95403F8449A
:1043D20010F582EEA2E292F0A2E092F1A2E392F252
:1043E200A2E192F3E5F0540FF0E576200205E575BF
:1043F200C4540FB50044D25C22B40E067710128961
:104402007922B40F0477068032B402028010B4031A
:1044120002800BB40A028006B40B02800122E95426
:1044220003F8E576200205E575C4540FB5000B903C
:10443200E8402582F582EEF0D27522E79097439309
:10444200B4040E90ED00E0A2E77404500D740380F2
:1044520009B45A0690ED00E0547FF8E9540312853E
:104462008F171289792290F41112838950117420C6
:10447200B152746BB152E8B13490F001128396904C
:0E448200F00112838950117420B1527463B19D
:1044900052E8B13490F40112839622E020E002C386
:1044A00022438203E0F8D322E030E2FC438203E8B7
:1044B000F0227583F0F830E3037583F4C40324011C
:1044C000F582E020E004C3E4800B5382F8438203CA
:1044D000E0128F16D3FE22A2E2924AC0E0917BD076
:1044E000E054039084A093C002FA128A517C0878A9
:1044F000009144E5C8304A02E5C05AC36001D3EEDA
:1045000013FEDCED9144E5C8304A02E5C05A600173
:104510000C9144E5C8304A02E5C05AC24A6002D252
:104520004AC39126E572F442C8E573F442C0128A88
:1045300026D002ECA2E0EE22C0E0400AE57252C8AA
:10454000E57352C0800AE572F442C8E573F442C0D4
:10455000D0E07F0180027F04DFFEC0E0E57052C83A
:10456000E57152C07F0EDFFEE570F442C8E571F4DC
:1045700042C0D265E570F4600855C88009C0E0808B
:10458000F1E571F455C07002C265D0E022FE2055FD
:104590000430190122A2E2C2E290849C937FFF4082
:1045A00001CFF57103F573CFF57003F57222F7FDB6
:1045B000DF7F040110407D00C0E0128F2A1284CBFF
:1045C000D0E05002DDF2222055063019030221ED21
:1045D000BE04005005128EEE8003128F02FFEEA281
:1045E000E2C2E290851C93400445C8800245C0CFDA
:1045F000BFFF028002D322128A5112846B30651EE3
:10460000C3128426306517A2D0B37C091312842606
:1046100030650BDCF7D3128426C3128A2622D3FC22
:10462000E572F442C8E573F442C0ECD380ECF3FCCD
:10463000CF3FC0E0740925748355D8D36001C3D03F
:10464000E02202010804300111C0E0C4540FB14956
:10465000D0E0C0E0540FB149D0E022B40A004002DB
:1046600024072430300107F5993099FDC299229032
:10467000E857E0D5E0027406F0B406247938E7B4D0
:10468000100280045403600FB24020400A770053A8
:1046900001F77700430108E52803F52809B940DE52
:1046A00022C8128F1BC890972993FAC3B1A87C081F
:1046B000E813B1A8DCFBD3B1A822CA858AF020F7A1
:1046C000FA858AF030F7FA400452C88004F442C8F0
:1046D000F48024C8128F20C8C3B1D57C08E813B178
:1046E000D5DCFBD3B1D522CA858AF020F7FA858ABA
:1046F000F030F7FAB392B2858AF020F7FA858AF0A3
:1047000030F7FA858AF020F7FA858AF030F7FACA8E
:1047100022C8128F1BC890972993FAC3D11C7C0919
:10472000E8A2D0B313D11CDCFBD3D11CC322CA85B1
:104730008AF020F5FA858AF030F5FA4006F442C88E
:10474000F4800252C8858AF020F5FA858AF030F5A7
:10475000FA858AF020F5FA858AF030F5FACA22AC9B
:104760007420020CE57554C07023E575C45403FC35
:1047700074382CF82404F9E6B41001225403700FA5
:10478000E7B4100122B434012254037002D322C3CF
:1047900022C320020DE57554C0700EE575C45403A4
:1047A0008002E576B50402D322C3227C0075A0E81E
:1047B0007880EC20021F12867F401890E930E0F5E7
:1047C000F0ECB578005003A4800BE578A42CC395D9
:1047D000788002E576F2080CBC04D722E9540390F5
:1047E00084A093FAE9A2E2E5C85002E5C0FE5A703F
:1047F00044EE035A603F5012E5C8FE5A7007EE03BC
:0E4800005A70028030E5C05A702BE9540771DF
:10480E00C5304A0F20D0045004800A50087433C2B9
:10481E004A80027422B93C005005128EF3800312B6
:10482E008F07304A0280030287B2E7B4100AE920EC
:10483E00E22CBEFF320287ECE930E2F912874FB468
:10484E00EEF3BEEC030287ECBEFF030287ECAC0670
:10485E00028806540390E87C2582F582E0221287B6
:10486E004FB4F303128988770DE920E2495403907F
:10487E00E840FC2582F582E0B4ED1FEE7583E98CED
:10488E0082438210F0D17F502DE07583E98C8243F4
:10489E008210F0D25C02884E8056B4F019EE701978
:1048AE00ECB5780085768240028C827583EAE054FE
:1048BE000323232416F70289071289675407B404C9
:1048CE0000501BEE30020D30E70AA2E45403B392FF
:1048DE00E4F0800AE054F05306034EC2E7F0D17FB5
:1048EE005070EEA2E79207C2E7E0F579D25D8062E2
:1048FE0090921F7C45B93C0040059092437C65A385
:10490E00A3ECB58250B465077CFEE954078012BE55
:10491E00FE19E954037CFAB5740790E885ECF0E5CE
:10492E007412847BEC1284B5028907128967B45520
:10493E0006EE1282F9801775A0E8E954032440F8B8
:10494E00E2F87429B8FE005014B8FB00400F740D45
:10495E00770D028907E493B506A5A3E493F7E9540E
:10496E0007A2E2C2E290E840500390E87C2582F56F
:10497E0082EEF0E9540730E271C2E2B57400BEF285
:10498E0019E95403B5780050057742028907128958
:10499E006754F07002773A028907D2E2BEE92475B5
:1049AE000504F5007C14E812847BE505240F83C012
:1049BE00041284B5D0045002DCECD505E9804C3CE1
:1049CE000390FA9092A5540393BEF404427D803B6B
:1049DE00BEF50B2018F82019F5F4527D802DBEFF80
:1049EE00EDC0E01289DFD0E080E9BEFF1E7583E9DD
:1049FE00E95403F582438210E4F012896754F044BF
:104A0E0002F0E95403FC12867F925CE7B434028014
:104A1E0004540360558B0006E6FEE7B40800500709
:104A2E009091D5936E7043E9A2E2E5C85002E5C0BD
:104A3E00035A7003168033E95403C074F57412855B
:104A4E0020D0744025E9540712847BE79091DD93C2
:104A5E00FCE95407B5740590E885ECF0EC1284B5CA
:104A6E0050031680051776003179227583E8E954D4
:104A7E00032480F582E07583EAF582E022E924CBF7
:104A8E0083522822FEFDFBF7EFDFBF7FBEC80280F8
:104A9E003CBE64081289CFB4C8318031BE502C128E
:104AAE0089CFB46426C3204D01D3C0D0128967D0FC
:104ABE00D0540F50024410FEE95403B57800400B59
:104ACE00CEF0CEFC12867F50028E797E001289D4F3
:104ADE00EEF0221289D4E02290E878E95403258280
:104AEE00F58222C006D31289A67E001289C9D0068D
:104AFE0022201835201932128520204E2C402AE50E
:104B0E0079B4440975F0FF78B6128F4C22B4550F64
:104B1E00E574780D12858FE574788D12858F22B429
:104B2E007707E57478B31280F42220022530AF2483
:104B3E00C0E0203B12E55F64446015E55F6455609C
:104B4E000FC289D2A8D2B2203A06C28BD2AAD2B351
:104B5E00D0E0D2A92220023530AF3430A816202F53
:104B6E00FD203B10C2A87CFF20B204DCFBD266C243
:0E4B7E00B275250830AA162037FD203A10C265
:104B8C00AA7CFF20B304DCFBD267C2B3752608C233
:104B9C00A922200236205E33205930205A2D20586D
:104BAC002A203D27205C24205D21203C1E205B1BFD
:104BBC00C3E5592410955A540FB40900500DE599CA
:104BCC00C298201207B43F0485769922F599309942
:104BDC00FDC29910124C205E48B40005D212C220BE
:104BEC0022B40105D212D22022F890E852E0C8B4C7
:104BFC000D1518E577B50000400A8876C270C238EA
:104C0C00D26FD215E4F02224D0B40A005013C8C0DD
:104C1C00F075F00AA4D0F030D2028005285001E4DF
:104C2C00F02220200AA850F60853006F885022A8C2
:104C3C0059F60853004F8859D249228556007553AE
:104C4C0000E579540FFE300205200705800C301862
:104C5C00097E03B4030050027E0275A0E87920BEE1
:104C6C000402801FB81A028003B89A17EE1423238B
:104C7C00FE909265755300EE936007F3090E055391
:104C8C0080F522E86007A2E792F0028BCBBE03030B
:104C9C00028C134011E557A2E792F0C2E7B4190059
:104CAC0040EEF8028C52E557B4050050E374E0F383
:104CBC0009755301E5571423255714F8909285BEB6
:104CCC000103909279E89360070553F3A30980F5EB
:104CDC0022BE0133E8547FB40F0C30F002803A90BE
:104CEC009291780080DF917A6009A2F092E7F375D7
:104CFC005301229092A974E0F309E8547F93A2F037
:104D0C0092E7F375530222BE0247E8547FB41F03A7
:104D1C00301806B40F0E30F00475530022909298A0
:104D2C00780080A1917A600F75530130F00674F011
:104D3C000553F309E8F32290932975530274E0F3B9
:104D4C000930F00974F00553F30953007FE893F32D
:104D5C0022BE0304917A80D0BE040491A28003BECB
:104D6C00051DE5567014B81905BE04AD8003BE05CB
:104D7C00A8909714E8C2E79361E4917A61E4222247
:104D8C00EE149093A9C0F075F080A424A9F582E5E7
:104D9C00F0D0F03493F583E8C2E793B4FF06D0E08B
:104DAC00D0E081136001F822B81A03D38004B89ABA
:104DBC0009C3D1A992E2F0D25C22B87C16D1A9D257
:104DCC005CB2E2F0D2F078FC30E207C2F0787C758D
:104DDC00530122B8FC06D0E0D0E08113B87B06D199
:104DEC00A9B2E18007B80E07D1A9B2E0D25CF022DB
:104DFC00D27375A0E87928E579C4540720192B20C3
:104E0C001823B40706D138755C0322B40406B12705
:104E1C00755C02224006B151755C0522B40206B1E4
:104E2C00F4755C03226003B1AF22B1B32290E82D7C
:104E3C00E0F5F0A3E0A2F492E6D2E790E829F09036
:104E4C00E82FE0A2F592E7F404A2E792E6A2F0B311
:104E5C0092E790E828F02290E82DE0F875F080F4C5
:104E6C00A2E092F2A2E192F0A2E292F1E5F090E8D7
:104E7C0028F088F0A2F490E82EE090E829B185A201
:104E8C00F590E82FE090E82AB18522401420E70441
:104E9C007800801B04F853007F7002787F747F8049
:104EAC000EB48000400478008005D2E7F87480F0DE
:104EBC00A3A3E8F022740380027404FCF55C90E870
:104ECC002D75A0E87828E0F208A3DCFA22A85A9005
:104EDC00E82D7C03E6F008A353004FDCF720021109
:104EEC00303908E57954F060088003204D03E480E4
:0E4EFC0002E608F053004F885A2290E82DE09D
:104F0A0075F040A2E092F5A2E192F4A2E492F1A235
:104F1A00E592F390E82EE0A2E692F0543F90E82959
:104F2A00F090E82FE0A2F392E7F404A2E692F2A24C
:104F3A00E792F3543F90E82AF090E828E5F0F0224F
:104F4A0090E82DE075F090A2E092F2A2E292F1A22E
:104F5A00E192F0A2E4B392F4A2E5B392F390E82EC0
:104F6A00E07002D2F430E702F40490E829F090E805
:104F7A002FE07002D2F330E702F40490E82AF090AE
:104F8A00E828E5F0F0222222E5795407B4040474F3
:104F9A007F80044017743068A2E7C2E7700EE57498
:104FAA00908EA5934004F452C02242C022080220E7
:104FBA0080E576200205E575C4540F4410F5827524
:104FCA0083E9E022751E748076751E738071751EE2
:104FDA0053806C751E6D8067751E2A8062751E2B44
:104FEA00805D751E798058751E7A8053751E6B8098
:104FFA004E751E4B8049751E638044751E43803F63
:10500A00751E78803A751E588035751E7080307509
:10501A001E50802B751E758026751E718021751E87
:10502A0051801C751E628017751E428012751E7291
:10503A00800D751E778008751E6D8003751E6E3093
:10504A000111C0E07420128552E51E128552D0E08B
:10505A0012853422C20DD20E30010CC8128F2FC80D
:10506A00C5F0128F2FC5F012912222D20DC20E3036
:10507A00010CC8128F34C8C5F0128F34C5F01291D2
:10508A002222C20843C83E7C0FDC02804D7DFFE528
:10509A00C8553C6004DDF880F07C000C0000E5C8CF
:1050AA00553C60F7C3EC9467500A20082D1291CC46
:1050BA00D20880D07C000CE5C8553C70F9C3EC944A
:1050CA0009500280157D08129096400E300903C3DC
:1050DA008001D3E833F8DDEFC322D322300A16E584
:1050EA003F52C8E53D52C07C68DCFEE53C42C0E563
:1050FA003E42C8C20A2200E8B42A06D20BD20C8069
:10510A004FC20BE854F3B42009300E3EC20ED20F40
:10511A00803AE854F3B43009300D2FC20DD20F8013
:10512A002BE854F3B4220A8EF08FE0C20ED20F801D
:10513A001B8017E8B42F0C75F06375E002C20ED21B
:10514A000F8009E8540FB40B0100C20F7C5FDCFE2C
:10515A00227D10C5F0D312906D00000000000000FF
:10516A003312906DBD0904C5F08003000000DDF024
:10517A00C312906D22C0E0E53F52C8E53D52C07CA3
:10518A000B500280027C19DCFEE53C42C0E53E423F
:10519A00C87C13500280027C06DCFED0E0227CFF31
:1051AA00DC028023E5C8553C70F67C000CE5C85546
:1051BA003C60F9C3EC9408500AC3EC94044008C25A
:1051CA00098002D209C322D322853C1E853D1D8552
:1051DA003E1C853F1B22851E3C851D3D851C3E8548
:1051EA001B3F227C26DCFE8015129096C2087CFFAB
:1051FA00E5C8553C6006DCF8D2088002C2082212D3
:10520A00909640257D08129096300903C38001D3F9
:10521A00EE33FEDDF17D08129096300903C380015A
:10522A00D3EF33FFDDF112909622888285F0831244
:10523A008A511290C11291A3128F7A402F12916B48
:10524A00300A028002800B128FD48582E08583F0B7
:10525A0080E6128FEE200B0E300F118582E08583D7
:10526A00F012904980061290DB1290F71290CE123B
:0E527A008A2622200D028003200E2DE854F01B
:10528800B400028021E854F0B42010E8B42E0302E0
:1052980091A0E8B42A028012200D0BE854F0B43033
:1052A80009200E028004D20A8002C20A22C082C0EB
:1052B80083E5749091C493F53C64FFF53DE57490E3
:1052C80091C893F53E64FFF53FD083D08222040154
:1052D80010400C0330C07C047DC8DDFEDCFA2200DF
:1052E8000A01000001030100AAFA000000AAFA005E
:1052F80083ABFA00FA000000FA00000000FA000090
:1053080001FA000002FA000003FA0000EE000000B3
:10531800FE000000BFB0FA00000008FA000000001C
:1053280003FA0000FC00000055FA00FF02F20BED42
:1053380011F311F40DF011F50DF60DF70DF80DF947
:105348000DFA0DFB0DFC0DFD0DEE25D229EF2FFFFB
:1053580007F60DF50DF40DF311F216E811E70DE659
:105368000DEA0DE900EC0DF00DEE0DEB34E43D3ADD
:10537800BA000058F0580014F0140000000000773C
:10538800F77F002A0000360000AA0000B6000012CD
:105398000000590000F01200F05900E11D45E19DA0
:1053A800C500E11477E1F014F0770004081020013B
:1053B8000240800000000000000000000000000023
:1053C800370000000000000000000000000000009E
:1053D8005D00000000000000000000000000000068
:1053E80000000000000000000000000000000000B5
:1053F80000000000000000000000000000001D0088
:10540800385B5C5253474F495148504B4D0035006B
:1054180000001C0000000000000000000000000068
:105428000000000000000000000000000000000074
:10543800004600000000000000000000000000001E
:105448007C000000000000000000000000000000D8
:105458002F00000000000000000000000000000015
:105468000000000000000000000000000000000034
:105478000000000000000000000000000000140010
:10548800111F2770716C697D7A75726B74004A0000
:1054980000005A00000000000000000000000000AA
:1054A80000000000000000000000000000000000F4
:1054B800007E00003B3C3D3E3F404142434457583C
:1054C8000046FF524F50514B4C4D474849FFFF563D
:1054D80000FFFF2BFFFFFFFFFFFFFFFFFFFFFFFFA7
:1054E800FF01290B02030405060708090A0C0D1A17
:1054F8001B2B2728333435390E0F1C2A361D00384C
:1055080000000000000000000000000000FF00375D
:105518004A4E00531E302E201221222317242526FE
:105528003231181910131F14162F112D152C453A46
:105538005400FF000506040C030B830A01097807D1
:10554800007EFF7069727A6B73746C757DFF6061A1
:105558000062625DFFFFFFFFFFFFFFFFFFFFFFFF2E
:10556800FF760E45161E26252E363D3E464E5554D0
:105578005B5D4C5241494A29660D5A125914001173
:1055880000000000000000000000000000FF007C98
:105598007B7900711C322123242B3433433B424B4B
:1055A8003A31444D152D1B2C3C2A1D22351A7758AB
:1055B8008400FF00070F171F272F373F474F565EFE
:1055C800575F627069727A6B73746C757DFF8013B4
:1055D8008D818153FFFFFFFFFFFFFFFFFFFF80FF6C
:1055E80082080E45161E26252E363D3E464E55543B
:0E55F8005B5C4C5241494A29660D5A1259110A
:105606005819398B8C67646E656F6D6360616AFFCC
:10561600777E847C79711C322123242B3433433BDF
:10562600424B3A31444D152D1B2C3C2A1D22351A6E
:105636007614FFFFFF007A78637660616264656DB9
:10564600676F696B7152535455565758595B5C399D
:10565600370A7F7F7F2AFFFFFFFFFFFFFFFFFFFF66
:10566600FFFFFF35321D1213141517161A1C191BCE
:1056760018211E2A29272B2F2C313330243838366F
:10568600363A3A37377275737774793E3D3B3C51FB
:105696004B434E454C41000B08020E0305042226DF
:1056A60028252E2D1F230C0F011120090D0710068A
:1056B6004739FFFF39000506080A0C0E10111207BC
:1056C600090B1617155E7071725B5C5D444546FFEB
:1056D600FF7C30303058FFFFFFFFFFFFFFFFFFFF6B
:1056E600FFFF7F1D2A271E1F20212223242526286F
:1056F6002940415856576B6C6D792B3559636E4C62
:1057060043130D787A2C42344A607B141B181CFF15
:105716002E2F477D5A324D68664F385051523D53B1
:1057260054556A693E3F36394E3A3C6737653B64A5
:105736006277FFFFFFFF565758595A5B5C5D5E5F05
:1057460060616263643A393F403E444542434AFFE2
:10575600FFFFFFFFFFFFFFFFFFFFFFFFFFFFFFFF53
:10576600FFFFFF06362D070D0E15161D1E25262ECC
:10577600353037382A312C3334523C08320504028E
:10578600555354FFFF653D666867695049484FFFAA
:105796006B6C4B6D51410A231B111012191A2721EC
:1057A60022292B24282F09170B18201C0F141F132E
:1057B6006A03FFFFFF00565758595A6465666768C3
:1057C600717281828392969798999A9B9D9E9FFF6C
:1057D600FFFFFFFFFF73747C7D80A0FFFFFFFFFFCD
:1057E600FFFFFFBFC9EFC0C5CBD0D6DBE0E5EAF9C6
:1057F600F5FAF6F7F2FBE8EDF3D4BCBEBDAEABAFFF
:10580600ADACB2B1FF888C8A8D8E8FAAA9A7A8FFEE
:10581600A2A3A4E89594C2D9CECDCCD2D8DDE6E237
:10582600E7ECE3DEEBF0C1D1C7D7E1D3C6C8DCC3F2
:10583600A1B0FFFFFFFBFEEFBF51762D020401036F
:10584600191A313348495F61300F7374757F6F00E1
:105856007F04FF005AFE000075B0FF75810775E8EA
:105866000475D8DF7590FCE4787FF6D8FDE590F4F2
:1058760054C02440F57F60FE74FFF5757550607561
:105886005160755940755A40757B00757C0090E8EB
:10589600577406F0D202129BA7B4E6FA129BA7FC35
:1058A60090ED00129BA7F0A3DCF9E57FC4FE90E91A
:1058B600107C04129BA7602AFF540CD2F0B5060296
:1058C600C2F0129BA720F0EBF0A3DCE77C04EFC448
:1058D600540FB4000590E92080D9B401D690EA00AF
:1058E60080D11280111280EA5389F0438901D28C4B
:1058F600D2A9D2AF437DC3306B03129B43306D09EF
:10590600E55C7005128E7EC26D12864D4003029ACA
:10591600F9E57BB57C02802775A0E8A87CE2F9E56D
:105926007412847BE91284B5500A0554E554B4A078
:105936000975540008B810027800887C029A7075C0
:10594600A0F47819E220E003029974781B20E5643C
:10595600E270030298E9B4FF22129935307BE91010
:10596600E612A95077000953016FF70953016F89B1
:0E5976005002996FF57EC264029949307BCAD7
:10598400F5F054FCB42822129935F975A0E8A87BE7
:1059940030F10574E012992D30F00574F012992D50
:1059A400E912992D887B02996FA950A7F009530138
:1059B4006F895002996F7C04A959781BE2FE307BF1
:1059C40033C3E5592410955A540FB40C0074804025
:1059D400027481129B90B4801BEE80097819E23026
:1059E400E0FC781BE2128534F70953014FDCED89A2
:1059F4005902996F029974129935A2E792235000C3
:105A0400F57E537E7FC264547FB401028013B430A8
:105A140002800EB403028009F85300F0B84015D296
:105A2400767819E230E0FC30E5030298A8781BE2AE
:105A3400F57AD264202320D27C8047F208B8100281
:105A44007800227819E230E0FC20E504781BE22299
:105A5400D0E0D0E00298A8307B2875A0E8A87B7439
:105A6400EF12992DE57E12992D30640F307607C21E
:105A74007674EF12992DE57A12992D887B74801231
:105A84009B90107C03029A70E57EB4012FC207E557
:105A94007AFE54F0B50614E57F6E54C0700DEEF531
:105AA400755430C4F576D26F029A6BC27B7575FF5C
:105AB4007576FF74AA42C0C2EC029A70B4160C74D4
:105AC40040B57FE77480129B9080E0B40309E57AC7
:105AD40090ED00F0029A70B43019E57AC454C0B560
:105AE4007F0EE57A54039092A593457DC57DD26DD2
:105AF400029A68F95301F0B94024F9C4657F54C08F
:105B0400701AE95403F9307B06B57403857A797504
:105B140083EA4400F582E57AF01280B78058B4092C
:105B240024207B028050128EA9F8129B38540FC493
:105B34004200C074857674128520D074B3E892E76D
:105B4400129B908039B40C07307B02D2EC8027B4CE
:105B54000208C2EC74AA42C0801CB43119307B1410
:105B6400E579540FB40400500BE574D2E212847B3F
:105B7400E41284B58000307B057480129B90306FF2
:105B840024E55C6015207209D27290E83FE4F0804D
:105B94001490E83FE0B40200400BC27285595A7574
:105BA4005C00129B6DE5537024E550B551028027CB
:105BB400A851E6F5560853006F700686570853003F
:105BC4006F8851128B35E553600D75552075A0E82B
:105BD400A855E2F81281C2307302800CE559B55A17
:105BE400028005128DC7D273E55C701130731812F0
:105BF4008CEAC273E55C600F755E28C27375A0E819
:105C0400A95EE3F812821F12814C105D14105C0629
:105C14001075210297EB128EA94490129B90029763
:105C2400EB129B38F85300070354384844C0129BC6
:105C3400900297EB7583E8E5744440F582E0547F65
:105C4400129B900297EB7583EAE5764400F582E0B7
:105C540022C26B12855D307B1B128520B3921B2000
:105C64001C05301B0F8003201B0AA21B921C74A06E
:105C740092E0719090E83FE004F0221289EDC26F47
:105C8400857674129B38F579128699E57444FCF58F
:105C940090D27BD2EC128520B3921B921C22C0E0DE
:105CA40075A0F47819E230E2FCD0E0781BF2300100
:105CB400031285522275A0F47819E230E0FC781BB7
:025CC400E222DA
:025CC6002D05AA
:025CC8006D4B22
:00000001FF
